:100000000C94F7040C9414050C9414050C9414052A
:100010000C9414050C9414050C9414050C941405FC
:100020000C9414050C9414050C946C190C94AE18D3
:100030000C948B200C9414050C9414050C9414054A
:100040000C9414050C9414050C9414050C941405CC
:100050000C9414050C943E200C9414050C94140577
:100060000C9414050C9414050C9414050C941405AC
:100070000C9414050C9414050C9414050C9414059C
:100080000C9414050C9414050C9414050C9414058C
:100090000C9414050C9414050C9414050C9414057C
:1000A0000C9414050C9414050C941405E1065507E2
:1000B000E906B306B706ED06BA06F006FB06C50666
:1000C0004B07C906FF06CD0603072D07D106070714
:1000D0003707D7060D071707BE06F406C106F70651
:1000E000DC061207230743074507AF06E5065E0750
:1000F0007E078407700678078A0790079607AF0780
:10010000D507DA07DF07E407E907EE07F307F80783
:10011000FD070208CA08CA08FD08FD087C099A09FB
:100120009B0A9B0A9F09130A240A240AFA0EFD0E51
:10013000380F5C0F630F6E0F710F710F710F8E1000
:100140008E10F60FF90FFD0F2210441047104A10C1
:100150006E10B916E0169618E01696182C174F1761
:100160009618451855184A1E401E581EAA1EAC1E49
:10017000AC1EAA1EAC1EAC1E791EAC1E831E8D1EAC
:10018000AC1EAC1EAC1EAC1EAA1EAC1EAC1EAA1E23
:10019000AC1E661EAC1EAC1E9D1E9D1E9D1E9D1E91
:1001A0009D1E9D1E9D1E9D1E9D1EA51EAC1E4A1EB3
:1001B0003D1EAC1EAC1EAC1EAC1EAC1EAC1EAC1E5E
:1001C000AC1EAC1EAC1EA51EAC1EAC1EAA1EAC1EE8
:1001D0009B1E9B1E9B1E9B1E9B1E9B1E9B1E9B1E57
:1001E0009B1EA51E00000000000000000000000093
:1001F00000000000000000000000000000000000FF
:1002000000000000000000007E0F00D4FFFFFFC7C9
:100210000000007800000000000000002A2B2800E9
:1002200000000000000000000000000000000029A5
:10023000000000002C1E3420212224342627252EE5
:10024000362D3738271E1F2021222324252633331D
:10025000362E37381F0405060708090A0B0C0D0E49
:100260000F101112131415161718191A1B1C1D2F15
:100270003130232D350405060708090A0B0C0D0E35
:100280000F101112131415161718191A1B1C1D2FF5
:100290003130354C1E0F0500047F3F1F643214645B
:1002A0003214783C1E1E140A050631FF0974A101A0
:1002B0000975150026FF00952075088102C005010B
:1002C0000902A10185020901A100050919012908F6
:1002D00015002501950875018102050109300931D4
:1002E0001581257F95027508810609381581257FBE
:1002F000950175088106050C0A38021581257F9540
:100300000175088106C0C005010980A10185031996
:10031000012AB700150126B700950175108100C0AC
:10032000050C0901A101850419012AA00215012665
:10033000A002950175108100C005010906A1018583
:1003400006050719E029E7150025019508750181C3
:10035000020507190029EF1500250195F0750181A7
:100360000205081901290595057501910295017588
:10037000039101C00660FF0961A101096215002611
:10038000FF009520750881020963150026FF00957E
:100390002075089102C005010906A101050719E0B1
:1003A00029E7150025019508750181029501750859
:1003B00081010507190029FF150026FF0095067524
:1003C0000881000508190129051500250195057505
:1003D000019102950175039101C0090274000401A5
:1003E00000A0FA0904000001030101000921110124
:1003F00000012244000705810308000109040100EF
:10040000020300000009211101000122220007055A
:1004100082032000010705030320000109040200F4
:10042000010300000009211101000122B6000705A7
:1004300084032000010904030001030000000921D6
:10044000110100012215000705850320000112019A
:100450000002000000085476610001000102000162
:10046000240330002D0053006900780074007900E7
:100470002D0075006E0064006500720067006C005E
:100480006F00770000001403760065006E003000F6
:100490006D007400720030006E0000000403090457
:1004A0002223252628292A2C2D2F30323335363881
:1004B0003A3B3D3E4042434547494A4C4E505153DA
:1004C0005557595A5C5E6062646668696B6D6F71FE
:1004D000737577797B7D7F81838587898A8C8E9000
:1004E000929496989A9C9E9FA1A3A5A7A8AAACAE09
:1004F000AFB1B3B4B6B8B9BBBCBEBFC1C2C3C5C649
:10050000C7C9CACBCCCDCED0D1D2D2D3D4D5D6D7F1
:10051000D7D8D9D9DADADBDBDBDCDCDCDCDCDDDD2F
:10052000DDDDDCDCDCDCDCDBDBDBDADAD9D9D8D71F
:10053000D7D6D5D4D3D2D2D1D0CECDCCCBCAC9C7C1
:10054000C6C5C3C2C1BFBEBCBBB9B8B6B4B3B1AFF8
:10055000AEACAAA8A7A5A3A19F9E9C9A9896949298
:10056000908E8C8A89878583817F7D7B797775736F
:10057000716F6D6B6968666462605E5C5A5957554D
:100580005351504E4C4A4947454342403E3D3B3A09
:100590003836353332302F2D2C2A29282625232290
:1005A00035001E001F00200021002200230024002F
:1005B0002500260027002A002B0014001A0008003E
:1005C000150017001C0018000C00120013004C004E
:1005D000290004001600070009000A000B000D00A6
:1005E0000E000F0033003400E1001D001B00060068
:1005F00019000500110010003600370038002800EF
:100600003900E000E200E30021522C002C002252CD
:100610005000510052004F0035021E021F022002FE
:1006200021022202230224022502260227022A0096
:1006300035021E021F02200221022202230224028E
:100640002502260227024C004C003A003B003C00E9
:100650003D003E003F002D022E022F0230023102EB
:1006600001004000410042004300440045003202C6
:1006700064024A004D000100010001000100010078
:100680000100010001002352AB00AA00A900AE0046
:1006900035001E001F00200021002200230024003E
:1006A0002500260027002A0035001E001F0020001C
:1006B00021002200230024002500260027004C00F2
:1006C0004C003A003B003C003D003E003F002D0046
:1006D0002E002F0030003100010040004100420098
:1006E000430044004500320064004B004E0001000E
:1006F000010001000100010023520100010001007E
:10070000AB00AA00A900AE003A003B003C003D004F
:100710003E003F00400041004200430044004500CD
:100720000100007C01000100010001000100010046
:1007300001000100010001000100010001000100B1
:1007400001000100010001000100010001000100A1
:100750000100010001000100010001000100010091
:100760000100010001000100010001000100010081
:100770000100010001000100010001000100010071
:100780000100010001000100010001000100010061
:100790000100010001000100010001000100010051
:1007A0000100010001000100010001000100010041
:1007B0000100010001000100010001000100010031
:1007C0000100010001000100010001000100010021
:1007D0000100010001000100010001000100010011
:1007E0000100010001000100010001000100010001
:1007F00001000100010001000100010001000100F1
:1008000001000100010001000100010001000100E0
:1008100001000100010001000100010001000100D0
:1008200001000100010001000100010001000100C0
:1008300001000100010001000100010001000100B0
:1008400001000100010001000100010001000100A0
:100850000100010001000100010001000100010090
:100860000100010001000100010001000100010080
:100870000100010001000100010001000100010070
:100880000100010001000100010001000100010060
:100890000100010001000100010001000100010050
:1008A0000100010001000100010001000100010040
:1008B0000100010001000100010001000100010030
:1008C0000100010001000100010001000100010020
:1008D0000100010001000100010001000100010010
:1008E00001000100010001000001010101010101FD
:1008F00001010202020202020202020303030303D5
:1009000003030304040404040404050505050506A3
:100910000606060607070707070808080809090961
:10092000090A0A0A0B0B0B0C0C0C0D0D0D0E0E0E0A
:100930000F0F0F101011111112121313141415159B
:1009400016161717181819191A1A1B1B1C1D1D1E0D
:100950001E1F202021222223242425262627282961
:10096000292A2B2C2D2D2E2F30313232333435368F
:100970003738393A3B3C3D3E3F404142434445468F
:100980004748494A4C4D4E4F50515354555658596B
:100990005A5B5D5E5F616264656668696B6C6D6F12
:1009A0007072737577787A7B7D7E80828385878885
:1009B0008A8C8E8F91939596989A9C9EA0A2A3A5BF
:1009C000A7A9ABADAFB1B3B5B7BABCBEC0C2C4C6C0
:1009D000C9CBCDCFD1D4D6D8DBDDDFE2E4E7E9EB7C
:1009E000EEF0F3F5F8FAFDFFFFAA7F554000112461
:1009F0001FBECFEFDAE0DEBFCDBF11E0A0E0B1E077
:100A0000EEE4FAE502C005900D92A03BB107D9F7DC
:100A100023E0A0EBB1E001C01D92A439B207E1F7D9
:100A20000E94F40A0C94252D0C940000A8E0B0E07C
:100A3000ECE1F5E00C949D2CFC018481882309F401
:100A4000CFC57F0121E04081518162817381958111
:100A50000E9485298C01F7019581992309F438C1F9
:100A6000980137572038310508F054C1003108F09B
:100A70003FC18FEF93E00E94842B811139C130E791
:100A8000A32E33E0B32E002379F0A114F4E0BF06C7
:100A900009F42EC1C5010E94842B811101C00150AF
:100AA0002FEFA21AB20AEFCFCE0101962C0188E0F7
:100AB000F20111928A95E9F72AE0322E85010F5F43
:100AC0001F4FC5010E94842B89831A82882309F451
:100AD0000FC1813009F041C06501F2E0CF0ED11C99
:100AE000C8010E94842B8A83882309F401C19FEFE7
:100AF000980F933060F423E0A20EB11CC6010E944F
:100B0000842B8B83882309F4F3C01C8229C0843092
:100B100031F54E0133E0830E911C02E010E05601E6
:100B20008FEFA81AB80AC6010E94842BF4018193A2
:100B30004F01882309F4DCC08C3741F4E2E0F0E097
:100B4000EC0FFD1FE00FF11F10820AC00F5F1F4F57
:100B500065010730110519F7CBC0580101C05601D6
:100B60008201F8012081222309F4A8CF213009F065
:100B700053C08181813081F46801F2E0CF0ED11C35
:100B8000F8018281893319F460E570E002C060E009
:100B900070E00E94BA1515C0823049F46801F2E095
:100BA000CF0ED11CF80182810E94C5140AC0833087
:100BB00051F46801F2E0CF0ED11CF80182810E944D
:100BC0006B14860182C0843019F00F5F1F4F7DC007
:100BD000F80122810E5F1F4F80E090E030E020534B
:100BE00031092A30310568F4389EA001399E500D34
:100BF0001124C901840F951F0F5F1F4FF801208139
:100C0000EDCF009709F461C0EFE9FFE03197F1F70C
:100C100000C000000197F5CFE22FF0E0EC5EFD4F41
:100C20002490822F86958695869590E0FC01EC5F56
:100C3000FD4F64902770712C022E02C0759467944A
:100C40000A94E2F7F1E06F227724FC01EC50FE4FAA
:100C50008490912C022E02C0959487940A94E2F716
:100C600031E083229924FC01EC51FE4FC490D12C39
:100C700002C0D594C7942A95E2F781E0C822DD240A
:100C80006114710419F081EE0E94C514811491045D
:100C900019F086EE0E94C51460E070E0822D0E947B
:100CA000BA158114910419F086EE0E946B14611438
:100CB000710419F081EE0E946B14C114D10429F063
:100CC00060E070E08CE20E94BA150F5F1F4F49CFC1
:100CD000F801E851FC47E730F10508F060C404C1B1
:100CE00006E221EE41EE6AE17CE7C7010E94AD21F8
:100CF00080912E02877009F473C4F70185818823DF
:100D000009F46EC48091560382FF6AC482E00E9497
:100D1000EC1366C4F801E851FC47E730F10508F42C
:100D2000E3C010924E03980130572332310508F08A
:100D300003C184E090E00E94922B9093560380932D
:100D40005503F801E150F047E232F10520F4EA5A88
:100D5000FF4F0C94812C809155038160ACC0809131
:100D600056038860B4C0809155038260A4C080910E
:100D7000550320C08091550388609DC08091560323
:100D80001EC0809156038260A2C08091550380618D
:100D900092C08091550380628EC08091550380641B
:100DA0008AC00E94291480915503806884C0809174
:100DB0005503886084607FC08091560382608160A3
:100DC00086C0809155038E7F76C080915603877FC1
:100DD0007EC0809155038D7F6EC08091550320C0E9
:100DE00080915503877F67C0809156031EC0809114
:100DF00056038D7F6CC0809155038F7E5CC08091BF
:100E000055038F7D58C0809155038F7B54C00E943D
:100E10002914809155038F774EC080915503877FA9
:100E20008B7F49C0809156038D7F8E7F50C080910B
:100E3000550382FB222720F991E0922790FB82F94B
:100E400090FB83F938C080915603982F909591704C
:100E50008E7F892B90FB81F93AC08091550386FBE8
:100E6000222720F991E0922790FB86F924C00E9466
:100E700029148091550387FB222720F991E09227BE
:100E800090FB87F918C061E001C060E08EE090E05F
:100E90000E94A82B1EC08091550384FB222720F9B5
:100EA00091E0922790FB84F906C080915503982F1A
:100EB000909590FB80F9809355030BC08091560369
:100EC00083FB222720F991E0922790FB83F98093FE
:100ED0005603609155037091560384E090E00E94A0
:100EE000C62B0E94291404CFE858FF4F0C94812C84
:100EF00007E225EE45EE6BE17CE7F7CE06E221EE58
:100F000040EE68E17CE7F1CE07E225EE44EE69E1D0
:100F10007CE7EBCE06E221EE42EE6CE17CE7E5CE2B
:100F200007E225EE46EE6DE17CE7DFCE08E221E048
:100F300045EE6EE17CE7D9CE809185030631FCE772
:100F40001F0709F420C38272F801E052F847EB3022
:100F5000F10508F05CC0E158FF4F0C94812C8091A2
:100F6000C20280FF19C0282F2E7F2093C202309129
:100F7000C3024091C4025091C5026091C6027091B3
:100F8000C7028091C8029091C9020E94EE27109278
:100F900093030E948927ACCE81608093C20261E0F6
:100FA000869586950E942229A3CE882329F00E9447
:100FB0006E299ECE8823D9F30E94792999CE882361
:100FC00029F00E940E2994CE8823D9F30E94182973
:100FD0008FCE882329F00E94F4288ACE8823D9F363
:100FE0000E94012985CE882329F00E94DA2880CE2C
:100FF0008823D9F30E94E7287BCE882329F00E941A
:10100000142876CE8823D9F30E942E2871CE073774
:10101000FCE71F0711F481E005C008372CE7120731
:1010200049F482E00E941A1443E062E081E00E94E9
:10103000BD135ECE9801205E324520323105A8F402
:10104000911115C00F7181E090E0FC0102C0EE0F1C
:10105000FF1F0A95E2F78F016E2F83E090E00E9458
:10106000A82B802F0E94261443CE9923E9F1033048
:10107000FCE71F0729F148F401153CE7130791F03D
:1010800001308CE7180711F12FC00B359CE71907C9
:1010900041F10C35ECE71E07E1F00A351C4721F55C
:1010A00081E020C00E9429142FEF34E38CE021500E
:1010B00030408040E1F700C000000E942D2018CE93
:1010C0006FEF7FEF80E090E00E94C62B0E943A2AEB
:1010D0000FCE8091560382FB882780F991E0892703
:1010E00001C080E00E940314F70185810081118115
:1010F000882349F0C8010E946B11D82E682FC801BF
:101100000E94851304C0C8010E945113D82EB80153
:101110008D2D0E94EB240E94F924D82E192FA82E81
:10112000F7010581C680C2949FE0C92280912E02FA
:10113000877001F10023F1F0812F807F803469F006
:1011400080E28D0D8830B0F0812F807E803229F4CE
:10115000F1E0FD1578F4CC2069F08091560382FF10
:1011600009C082E00E94EC1380912E028770BB249C
:10117000B3948111B12C912E92948FE09822892DF5
:1011800090E08C30910508F0D6C1FC01E657FF4F86
:101190000C94812C812F807F1F70882311F0129571
:1011A000107F0023B9F0112309F4B3C180E28D0D43
:1011B000883010F0A11006C090918503192B109370
:1011C000850305C090913002192B109330020E94C4
:1011D000AE269FC18D2D0E946B14112309F4ABC163
:1011E00080E28D0D883088F1AA2079F110959091D8
:1011F00030021923109330022BC0812F807F1F7083
:10120000803211F01295107F8D2DAA2029F021E057
:10121000A21609F44CC057C08091560382FD1BC032
:10122000002369F0112339F090918503192B109355
:1012300085030E94AE2680E00E94C5147CC180E038
:101240000E946B14112309F476C1812F0E94A726F6
:101250000E94AE2670C1002381F0CC20C1F131E0A4
:10126000C31269C190912F02812F8923181709F4A5
:1012700062C1192B10932F025EC1C1105CC1812F76
:101280000E945A1480912F02912F982329F0912FB8
:101290009095892380932F022091B301812F82237F
:1012A00009F449C1109521232093B30144C10023BF
:1012B00029F085E08C1508F43EC109C094E09C1526
:1012C00008F439C115C0002331F0C11022C1812FAB
:1012D0000E94611430C1CC2059F0893309F028C133
:1012E000EFEFF7EE23E0E150F0402040E1F71EC1C0
:1012F000812F0E945A141FC1812F86958695837075
:1013000019F0813061F017C1002321F08D2D912F4C
:10131000937002C080E090E00E943E2112C1002341
:1013200021F08D2D912F937002C080E090E00E94FB
:10133000192107C1602F8D2D0E94502A02C1812FD3
:101340008370A9F50111FBC04D2D4295469547705C
:10135000440F440F8D2D8F7090E09C01042E01C02E
:10136000220F0A94EAF7D4FE08C08FE090E001C093
:10137000880F4A95EAF7809501C080E0169516958A
:101380001370123069F088F490918603113019F0CF
:10139000822B892302C0922B892B0E942614CFC056
:1013A000822B909186038927F8CF822BF6CF0023DA
:1013B00019F0812F817001C08695882309F4BFC080
:1013C0004D2D429546954770440F440F8D2D8F70DB
:1013D00090E09C01042E01C0220F0A94EAF7D4FE8B
:1013E00008C08FE090E001C0880F4A95EAF7809529
:1013F00001C080E0169516951370123059F078F4FC
:101400009091BE01113019F0822B892309C0922BD3
:10141000892B06C0822B9091BE01892701C0822BA7
:101420000E94BA138CC01F70002339F0812F0E94D4
:101430001A148D2D0E94611482C08D2D0E945A14A1
:10144000812F0E94DF137BC08D2D32EFA31681F117
:101450003A1538F090EFA91659F0E1EFAE1619F1F0
:1014600054C0F3EFAF1659F124EFA216C1F04DC0EE
:10147000002381F034E03C1508F45DC01F7181E069
:1014800090E0012E01C0880F0A94EAF79091BE0106
:1014900089271EC085E08C1508F44DC0EFCF8091E0
:1014A000560382FD1AC0002329F0812F8F7120C0BE
:1014B0000023D9F3812F8F710E94DF133CC00023DA
:1014C00051F01F7181E0012E01C0880F0A94EAF7E4
:1014D0000E94BA1330C080E0FBCF002361F0812F5F
:1014E0008F7198E0899F90011124236020932E0230
:1014F0000E941A1420C081E00E94EC13E1E0EC1578
:10150000D0F482E00E94EC1316C0002321F0CC201E
:1015100061F28D2D91CECC2069F2893349F4FFEF31
:1015200027EE33E0F15020403040E1F700C00000EA
:101530008D2D0E946B1488EF890D843010F40E9469
:101540006321BB20A9F080912E0280FD11C0F7011C
:1015500015828695869586950E941A14C7010E9469
:10156000160580912E028695869586950E94DF133A
:1015700020E0F701408151816281738184819581EE
:101580000E9485292DC08A7A91E009F490E0909319
:10159000B201811112C089E20E94E2200BC0063123
:1015A0002CE7120771F48091B201811108C089E221
:1015B0000E94B4200E94AE269BCB85E3EDCF85E34D
:1015C000F7CF07373CE7130711F481E006C008376F
:1015D0008CE7180709F02ECD82E00E94DF1324CD9E
:1015E0002896E2E10C94B92CA6E2B0E0EAEFFAE02A
:1015F0000C949D2C85B7806885BF85B7806885BFB2
:1016000084B7877F84BF0FB6F894A8958091600057
:10161000886180936000109260000FBE90E080E8C7
:101620000FB6F89480936100909361000FBE81E043
:101630008093110181EB9EE19093B1018093B00101
:101640000E94F2180E9411198091E2008460809338
:10165000E200789480913E028823A1F01091E90085
:101660001F709091EC00892F817090FD80E8182BFD
:101670001092E9008091E80083FD0E94D2151F704E
:101680001093E90082E084BD93E095BD9AEF97BD89
:1016900080936E000E949421811102C00E94262333
:1016A00006E211E09BE2E92E91E0F92ED8018D913E
:1016B0008D018F3F11F00E942124E016F106B1F751
:1016C0000BE211E087E3E82E81E0F82EF80181912A
:1016D0008F018F3F11F00E942124E016F106B1F72F
:1016E0008AE0EBECF1E0DF01282F1D922A95E9F763
:1016F000E4EBF1E0DF011D928A95E9F780E090E0EC
:101700000E94922B853E9E4F21F40E9494218111CC
:1017100002C00E943A2682E090E00E94842B8093CF
:10172000130384E090E00E94922B909356038093E1
:1017300055030E943824EFEFF6E721E0E150F04036
:101740002040E1F700C000000E9438248091CB01C6
:1017500080FF08C06FEF7FEF80E090E00E94C62B13
:101760000E942D2083E090E00E94842B0E9426148A
:101770008091BF01811180C088E090E00E948C2B95
:101780004B015C0183E290E00E94842B282F30E023
:1017900040E050E060E070E080E090E000E20E9415
:1017A000D42C282939294A295B292093C202309355
:1017B000C3024093C4025093C5026093C602709363
:1017C000C7028093C8029093C9022C7F09F042C0DF
:1017D00025E02093C2021092C3023FEF3093C4026F
:1017E00039EB3093C5021092C60230E04FEF59EB4F
:1017F00060E00E94EE2788E090E00E948C2B6B0155
:101800007C0183E290E00E94842B282F30E040E0AE
:1018100050E060E070E080E090E00E94D42CB22FB5
:10182000A32FF42FE52F5B0197018601BC29A12B83
:10183000F22BE32BB093C202A093C302F093C40235
:10184000E093C5026093C602B092C7028093C802BB
:101850009093C9020E94D327109293030E94D11A39
:101860008091C20280FF05C060E0869586950E9447
:10187000222981E08093BF0184E091E0909352039C
:101880008093510344244394222423948E010F5FB8
:101890001F4F80913E02853009F041C0B0E4FB2E1D
:1018A00080913E02853009F036C080913E0284303E
:1018B00019F11092570388E190E00FB6F894A895BB
:1018C000809360000FBEF092600083B7817F8460D8
:1018D00083BF83B7816083BF7894889583B78E7FF9
:1018E00083BF0FB6F894A8958091600088618093BB
:1018F0006000109260000FBE0E943824EBECF1E013
:1019000081919191892B09F012C4A5EDB1E0AE1738
:10191000BF07B1F7C5CF0E9429140E9463210E941E
:101920003824F0ECEF2EF1E0FF2EABEC6A2EA1E0B4
:101930007A2ED301F701219131918D919D918227CA
:10194000932721E0EA3CF20719F0892BA1F305C0A7
:10195000892B19F40E9416263EC0512CD3018D907C
:101960009D903D01F701A080B180A824B924A11465
:10197000B10441F1312CCC24C394D12CC6018A216D
:101980009B21892BB1F039A25AA20E947F209CA3EF
:101990008BA32DA291E0960128213921232B09F454
:1019A00090E09EA349A15AA16BA17CA18DA10E94A8
:1019B000AA293394CC0CDD1CFCE03F12DFCFD70109
:1019C0008D929C925394B2E0EB0EF11CE5E05E1216
:1019D000C5CF0E94732080919303882309F4ABC084
:1019E00080919203E091C202E695E695E81BE093B0
:1019F0008E03823059F4F0E0EB55FD4FE491EE2E6A
:101A0000F12C66E4C62E6DE1D62E70C0863059F4F6
:101A1000F0E0EE55FD4FE491EE2EF12C56E3C52E8D
:101A20005DE1D52E63C0893061F4E695F0E0E156C2
:101A3000FD4FE491EE2EF12C4EEEC42E4CE1D42E4F
:101A400055C08F3061F4E695F0E0E456FD4FE49127
:101A5000EE2EF12C3AE8C32E3CE1D32E47C085315F
:101A600059F4F0E0E756FD4FE491EE2EF12C2BE314
:101A7000C22E2CE1D22E3AC08831F9F0833249F4DB
:101A8000E7E9F2E0E590F49099E1C92E9DE1D92EC5
:101A90002DC08432D1F0853209F58E2F63E00E948B
:101AA0003F2CE92FF0E0EC56FD4FE491EE2EF12CA7
:101AB00089EFC82E8AE1D82E19C0A8E2EA2EF12CAF
:101AC000B0ECCB2EBBE1DB2E11C0E4EFEE2EFF24F9
:101AD000F394FEE8CF2EFBE1DF2E08C060EDE62E8A
:101AE00067E0F62E73EDC72E7AE1D72E80918F0333
:101AF000882361F010928F030E947F2090938D03C2
:101B000080938C0310929103109290030E947F2087
:101B1000E0918C03F0918D038E1B9F0B8F3F9F47AD
:101B200050F4EE0EFF1EF0928D03E0928C038CE8D1
:101B300093E0F601099586E0E6E4F3E0D801019030
:101B40000D928A95E1F7B0904703F0904803D0904A
:101B50004903C0904A03E0904B031092480310924F
:101B6000490310924A0310924B03F11003C0DD2089
:101B700009F458C080914403909145030E94642069
:101B8000AC0190913F03992339F02091150130E089
:101B90002417350758F046C020911601FAE02F9F10
:101BA000900111242417350718F03CC09F3F19F00D
:101BB0009F5F90933F03FF2061F00E9494221F14C7
:101BC00014F491E001C09FEF899F802D1124809330
:101BD0004803DD2061F00E9494221D1414F09FEF51
:101BE00001C091E0899F802D112480934903809149
:101BF00048038823B9F0A0904903AA2099F00E94D5
:101C0000D322882319F08093480302C040924803EE
:101C10008A2D0E94D322882319F08093490302C0A1
:101C200040924903C11003C0EE2009F44BC08091DB
:101C30004203909143030E9464209C0190914003D1
:101C4000992309F49AC221353105E0F19F3F19F03B
:101C50009F5F90934003CC2061F00E945B221C1494
:101C600014F491E001C09FEF899F802D112480938F
:101C70004A03EE2061F00E945B221E1414F09FEFD5
:101C800001C091E0899F802D112480934B038091A6
:101C90004A038823B9F0A0904B03AA2099F00E9430
:101CA000D322882319F080934A0302C040924A034A
:101CB0008A2D0E94D322882319F080934B0302C0FF
:101CC00040924B03809147038B111AC080914803C7
:101CD000882311F08F1114C080914903882311F0DB
:101CE0008D110EC080914B03882311F08E1108C016
:101CF00090914A03992331F081E09C1104C002C005
:101D000081E001C080E080FD15C080914803811111
:101D10000FC08091490381110BC080914A0381114A
:101D200007C081E090914B03911103C080E001C096
:101D300081E080FD0E943122BA82FB82DC82CD826A
:101D4000EE8286E0F801A6E4B3E001900D928A9558
:101D5000E1F70E9463219091CA01891721F08093D5
:101D6000CA010E94732080913E02843009F091CD17
:101D700083E08093E9008091E80082FF8ACD809122
:101D8000E80085FF21C00E94921A81111BC050E219
:101D9000C52ED12C780109C08091F100D7018D9317
:101DA0007D01B1E0CB1AD10869F08091E80085FD92
:101DB000F3CF8091E8008B778093E8000E94921A1D
:101DC000882399F391E001C090E08091E8008B773F
:101DD0008093E800992309F45CCD2981822F90E05B
:101DE000FC013197E331F10508F098C1EA56FF4F45
:101DF0000C94812C1A828CE0FEC08A81823009F416
:101E0000B3C150F4813009F089C10E9473209B83D3
:101E10008C837D836E8384C1833041F0843009F0EC
:101E20007DC11B821C821D821E827AC16B81D801FA
:101E300080E090E0262F30E0A901480F591F45307F
:101E4000510508F06DC1E62FE80FF0E0EE0FFF1F1F
:101E5000E553FE4F4081518113965C93139714967E
:101E60004C931497019612968E30910529F758C11C
:101E70008A81823019F0853051F050C16B817C81AC
:101E80008D819E810E94872C0E94702149C1809182
:101E9000C20280FF0AC08091C2028E7F8093C2027C
:101EA000109293030E9489273BC181608093C202F4
:101EB00060E08695869551C04C816B818A810E9435
:101EC000811D9D8358C12D813E81322723273227D2
:101ED0004C816B818A810E945A1D22C10E94F1228D
:101EE0001FC18A81823009F019C1283009F43FC02E
:101EF000293009F468C08B818230F9F098F4813080
:101F000009F00EC18C81E9EB8E9FC00111246FEFA7
:101F100070E00E94592C462F20E06091C40280910D
:101F2000C30222C08330E1F0843009F0F9C020E020
:101F30004091C5026D818C8117C08C81882309F482
:101F4000AACF8091C20281608093C20260E0869530
:101F500086950E94222960E08C810E942229E0C09F
:101F60008C818093C602DCC00E945728D9C08B8127
:101F70008230E1F078F4813009F0D2C08091C5025E
:101F8000FFEF8F9FC001112469EB70E00E94592C74
:101F90006C83C6C0833099F0843009F0C1C0809151
:101FA000C3028C838091C4028D83BAC08091C20227
:101FB00080FF03C08695869504C080E002C08091B2
:101FC000C6028C83ADC02091C2023091C302409101
:101FD000C4025091C5026091C6027091C7028091FF
:101FE000C8029091C9020E94EE279AC020E12A837C
:101FF00097C01A8280E98B8393C0EA80FB80FE241D
:10200000EF24FE24CC80D12C5801C70180599C4F6D
:102010009501201B310B2C153D0508F081C0A0E96E
:10202000EA16F10428F40E94842BF501848303C08E
:10203000D50114961C92BFEFEB1AFB0AEFEFAE1A14
:10204000BE0AE3CFEA80FB80FE24EF24FE24CC808E
:10205000D12C5801C70180599C4F9501201B310B91
:102060002C153D0508F05CC0F0E9EF16F10428F4EA
:10207000D50114966C910E94A82BBFEFEB1AFB0AB6
:10208000EFEFAE1ABE0AE6CF0E94E12249C087E018
:102090008A8346C0EA80FB80FE24EF24FE24CC80A5
:1020A000D12C5801C70188969501201B310B2C15A6
:1020B0003D05B0F5F8E4EF16F3E0FF0630F40E94BA
:1020C000842BD50114968C9302C0F5011482FFEF86
:1020D000EF1AFF0A2FEFA21AB20AE4CFEA80FB80C0
:1020E000FE24EF24FE24CC80D12C5801C701889611
:1020F0009501201B310B2C153D0590F4A8E4EA1640
:10210000A3E0FA0620F4F50164810E94A82BFFEFFA
:10211000EF1AFF0A2FEFA21AB20AE8CF8FEF8983D6
:1021200040E250E0B80182E00E94C61FB2CB80912D
:102130003D02882309F4B4CBB0E1B9BDE2E1E9BDC9
:1021400009B400FEFDCF8091D8008F7D8093D80028
:102150008091E00082608093E0008091E00081FD4A
:10216000FCCF0E9429149CCB87E290E00E94842B34
:102170001B821C821D828E83D3CF2B30310508F049
:1021800067CDA0CD20912D029091F40157E0291741
:10219000A9F030E0529FF001539FF00D1124EB5055
:1021A000FE4F7181761306C07081781303C075816C
:1021B000741306C02F5F3F4F2770E9CF80E008956A
:1021C00081E008959091850380913002892B909150
:1021D0002F029923E1F0892B90911001913041F465
:1021E0009091550397FF04C09EE121E233E003C0C4
:1021F00096E029E133E0F90120E0915028F0319197
:102200003323D9F32F5FF9CF211110922F020895B4
:1022100080912D029091F401891719F08F5F8770DA
:10222000FBCF0895CF93DF938091F30182958F7058
:1022300009F04EC08091F201882309F449C08091D1
:102240002D024091F4015091EE016091ED01C09199
:10225000EF01D091F00177E08417D1F190E0789F01
:10226000F001799FF00D1124DF01AB50BE4F1496A1
:102270002C911497222349F111962C911197251333
:1022800024C02C91261321C015962C91159721114D
:102290001CC012962D913C9113972C1B3D0B283C92
:1022A000310598F48091F3018F7080618093F30180
:1022B000E550FE4F80818F70806180838DEE91E0CC
:1022C0000E9416050E94081103C001968770C4CFB2
:1022D000DF91CF910895CF92DF92FF920F931F93DA
:1022E000CF93DF936C010091BE0180918603082B90
:1022F000C6E0D0E010E0C8010C2E02C0959587958D
:102300000A94E2F780FD04C02197A8F7F12C09C0D8
:10231000FC2EB6018C2F0E94EB240E94F924019719
:1023200099F38F2DDF91CF911F910F91FF90DF9047
:10233000CF900895CF93DF93EC010E946B11BE0103
:102340000E94EB240E94F924DF91CF910895FC01B3
:1023500024812223D9F0808191810E949A11929543
:102360009F70963079F010F4925001C09A509230DC
:1023700068F4803F69F018F4883E40F409C0843F57
:1023800029F406C0883E20F0813F11F080E00895D6
:1023900081E00895A4E1B0E0E0EDF1E10C94A32C1C
:1023A0008C0186E0F801DE011F9601900D928A955E
:1023B000E1F7F8018481E5809DEE892E91E0992E68
:1023C0009091F101911120C0882309F463C1EE209E
:1023D00009F442C0C8010E94A711F82E8823E1F138
:1023E00087E0F801D40101900D928A95E1F7809180
:1023F000F101813031F48091ED019091EE010E9464
:102400009A110E94121148C1F801D080C180A280A7
:10241000B380F090F2012091EF013091F001FF20A4
:1024200009F4E7C0A501421B530B483C510508F0D5
:102430009DC0882309F430C18091F301282F207FAB
:102440009091EE01222361F09C1509F460C0C8014F
:102450000E94A711811163C0C8010E9416051AC10C
:102460009C1113C09091ED019D110FC0E1100DC0A2
:102470008F7080618093F3018DEE91E00E941605CC
:102480008091F301F801868303C1E1103AC040E076
:102490006C2D8D2D0E94C21040E06C2D8D2D0E9460
:1024A000C210E82E8111F4C0DF86C88A8F85988912
:1024B0000E949A11292F22952F70243020F49F70AA
:1024C000223028F009C02A50223080F014C099230D
:1024D00049F0811107C013C0992321F0F8019681BA
:1024E000907F69F0805E883030F409C0803F38F01A
:1024F000815F833020F0C8010E941605EF2CFE2C6E
:10250000CBC08091F30181608093F301C1C09091B1
:10251000ED019D119CCFE1109ACFF80198C0EE20FB
:1025200009F49ACF2091F301822F82958F7090E069
:1025300002978CF08091ED019091EE019987888748
:10254000BB86AA868091F1018C871D862E87CE01DD
:1025500008960E94160587E0F801ADEEB1E0019003
:102560000D928A95E1F70E94121194C09091F301A7
:10257000292F207F51F48DEE91E00E94160587E00F
:10258000F40111928A95E9F783C0882309F484C085
:102590008091EE018C110CC08091ED018D1108C06D
:1025A000E11006C0F8019683C8010E9416056AC0B2
:1025B000C8010E94A711882309F44ECFEE2009F428
:1025C0004BCF2091F301822F82958F7090E002977C
:1025D00014F28091ED019091EE019A838983BC827F
:1025E000AB828091F1018D831E822F83CE010196F3
:1025F000B0CFA21AB30AF8ECAF16B10408F042C08B
:10260000882309F447C0FE2CEE2009F425CF8091E1
:10261000EE018C1129C08091ED018D1125C09091A2
:10262000F30190FD18C0892F82958F70282F30E01C
:102630002115310581F0F80196832F30310541F0E5
:102640008F5F982F9295907F86818F70892B8683DC
:10265000C8010E94160587E0F801ADEEB1E00190D7
:102660000D928A95E1F718C0C8010E94A711811147
:1026700072CF8091F30181608093F301C8010E94C1
:1026800016050AC087E0F40111928A95E9F704C0A3
:10269000F12C02C0FF24F3948F2D6496ECE00C948F
:1026A000BF2C292F953078F58C3068F590E03CE010
:1026B000239F800D911D1124682F677023E096954C
:1026C00087952A95E1F7FC01EE0FFF1FE80FF91F30
:1026D000EB52FE4F40E050E080E0219130E0062ECA
:1026E00002C0369527950A94E2F721703327042E0D
:1026F00001C0220F0A94EAF7822B4F5F5F4F4330ED
:10270000510559F7089580E00895292F953088F5EF
:102710008C3078F590E03CE0239F800D911D1124D2
:10272000282F277051E001C0550F2A95EAF723E0C2
:10273000969587952A95E1F7FC01EE0FFF1FE80FAC
:10274000F91FEB52FE4F20E030E070E04081CB01FA
:10275000022E02C0969587950A94E2F781708195C2
:1027600084278523842781932F5F3F4F23303105B2
:1027700069F708958093BE0108959091BE0121E00C
:1027800030E0F90101C0EE0F8A95EAF7D90102C0E5
:10279000AA0FBB1F6A95E2F7BD016E2B01C0220F85
:1027A0004A95EAF7892F8623681303C0892F822B65
:1027B00003C02095822F89230E94BA13089521E037
:1027C00030E001C0220F8A95EAF720958091BE0182
:1027D00082230E94BA13089590912E028095892336
:1027E00080932E02282F277069F4981759F0909142
:1027F000560392FF07C08695869586950E94DF1343
:1028000010922E0208959091560392FB222720F9F0
:10281000281779F080FB92F9909356036091550345
:102820007091560384E090E00E94C62B82E00E94E3
:10283000EC13089521E030E001C0220F8A95EAF7F9
:102840008091BE01822B0E94BA1308958093860363
:1028500008951092850380911001813041F4809198
:10286000550387FF04C08EE1E1E2F3E003C086E098
:10287000E9E1F3E0DF011D928A95E9F780E090E05D
:102880000E943E2180E090E00E94192110923002C7
:102890000E94AE26E6E4F3E086E0DF011D928A9511
:1028A000E9F710923F0310924003109241030E94F7
:1028B00031220895882321F00E94A7260E94AE2687
:1028C0000895882339F090918503892B809385039F
:1028D0000E94AE260895882309F456C0823859F420
:1028E0000E94632181FF50C089E30E94E2200E9480
:1028F000AE2689E30CC0833879F40E94632180FFFF
:1029000043C083E50E94E2200E94AE2683E50E9438
:10291000B4200E94AE260895843859F40E946321A1
:1029200082FF32C087E40E94E2200E94AE2687E444
:10293000EECF9CEF980F913A50F390E2980F9830B9
:1029400050F4877091E001C0990F8A95EAF7892FBA
:102950000E94A726DECF9BE5980F933028F480E0F5
:1029600090E00E943E21089598E5980F9B3128F44D
:1029700080E090E00E941921089593E3980F93312D
:1029800018F460E00E94502A0895CF93882309F438
:10299000EFC0C82F8238A1F40E94632181FDE8C0F6
:1029A00089E30E94E2200E94AE262FEF87EE93E09B
:1029B000215080409040E1F700C0000089E315C03D
:1029C0008338C1F40E94632180FDD2C083E50E9458
:1029D000E2200E94AE262FEF81EE94E0215080404D
:1029E0009040E1F700C0000083E50E94B4200E94FF
:1029F000AE26BEC08438A1F40E94632182FDB8C017
:102A000087E40E94E2200E94AE262FEF81EE94E040
:102A1000215080409040E1F700C0000087E4E5CFFE
:102A20008CEF8C0F813AA0F580911203813081F0F8
:102A300030F0823051F58C2F0E94AF1D99C08091EB
:102A40008503823209F060C08C2F0E94311E5AC06B
:102A5000809185038232C1F3C431A1F068F4CB3098
:102A600009F44EC0C03109F048C082E080931203DF
:102A700088E30E94AF1D44C0C93221F0C83309F475
:102A80003FC03BC01092120338C0109212033CC0EA
:102A900080E28C0F883068F4C77081E090E001C05C
:102AA000880FCA95EAF790918503892B8093850357
:102AB0009ECFEBE5EC0FE33040F4F0E0E55BFE4F3A
:102AC000808190E00E943E2153C0E8E5EC0FEB319D
:102AD00050F4F0E0EE0FFF1FE25BFE4F808191812A
:102AE0000E94192145C083E38C0F833108F040C058
:102AF00061E08C2F0E94502A3BC080E0817002C0B0
:102B000081E0FCCF811134C0809110018130E1F46B
:102B10008091550387FF18C0EC2FE695E695E69562
:102B2000F0E0E15EFC4F8281282F30E04C2F4770AF
:102B300081E090E002C0880F991F4A95E2F7822356
:102B40009323892B61F410C0E9E1F3E08FE193E076
:102B50002191C21721F08E179F07D1F705C08C2F46
:102B60000E94B4200E94AE268C2F0E94E2203FCF0C
:102B7000CF9108951F93CF93DF93182FEB010E94FD
:102B8000C514209741F08FE99FE00197F1F700C04D
:102B900000002197F6CF812F0E946B14DF91CF9117
:102BA0001F910895AAE2B0E0E8EDF5E10C94AC2C99
:102BB000E0E4F2E08091F100819342E0E834F40730
:102BC000C9F780914102833009F463C030F4813049
:102BD00071F0823009F4A2C0B9C08A3009F48EC005
:102BE0008B3009F46EC0893009F0B0C020C08091EC
:102BF0004002813A09F0AAC08091E800877F809363
:102C0000E8008091440290914502892B21F468E00C
:102C100084E392E003C060E080E090E070E00E9416
:102C2000681F8091E8008B778093E8008FC08091C7
:102C30004002813209F08AC080914402909145029D
:102C4000009719F0029709F081C08091E800877F12
:102C50008093E8008091E80082FD05C080913E02EB
:102C60008111F8CF73C02091F3008091F20090E0C1
:102C7000922B029731F48091F100813011F086306F
:102C800021F48091F10080930F018091E8008B770F
:102C900059C080914002813A09F058C080914402A5
:102CA00090914502892B09F051C08091E800877FFF
:102CB0008093E8008091E80080FFFCCF80911001B4
:102CC0003CC080914002813209F040C080914402B2
:102CD00090914502892BD1F58091E800877F809300
:102CE000E8000E94141F81E090914202911101C0FE
:102CF00080E0809310010E94291428C08091400236
:102D0000813221F58091E800877F8093E8000E945E
:102D1000141F8091430280930E0118C080914002DD
:102D2000813AA1F48091E800877F8093E800809148
:102D3000E80080FFFCCF80910E018093F10080912C
:102D4000E8008E778093E8000E94141F8091E800CD
:102D500083FFECC18091400290914102492F50E0E5
:102D60004A30510508F0E2C1FA01E755FF4F0C94D3
:102D7000812C803821F0823809F0D8C108C08091B8
:102D80003C0290913D02992389F082600FC08091AE
:102D900044028F70873008F0C9C18093E9008091A8
:102DA000EB0085FB882780F91092E9009091E800FC
:102DB000977F9093E8008093F1001092F10071C129
:102DC000282F2D7F09F0B2C1882319F0823061F0DD
:102DD000ADC180914202813009F0A8C1933009F061
:102DE00080E080933D022EC08091420281112AC072
:102DF000809144028F702FEF280F263008F096C183
:102E00008093E9002091EB0020FF1CC0933021F457
:102E10008091EB00806214C09091EB0090619093E0
:102E2000EB0021E030E0A90102C0440F551F8A9554
:102E3000E2F74093EA001092EA008091EB0088608C
:102E40008093EB001092E9008091E800877F8093E7
:102E5000E8000E94141F6AC1811168C110914202EA
:102E60001F778091E3008078812B8093E30080912D
:102E7000E800877F8093E8000E94141F8091E8009B
:102E800080FFFCCF8091E30080688093E300111104
:102E900002C082E001C083E080933E0247C18058B7
:102EA000823008F043C120914202309143022C3D10
:102EB00053E0350779F583E08A838AE289834FB747
:102EC000F894DE01139620E03EE051E2E32FF0E0BB
:102ED00050935700E49120FF03C0E295EF703F5FED
:102EE000EF708E2F90E0EA3010F0C79601C0C096C8
:102EF0008D939D932F5F243149F74FBF8091E80058
:102F0000877F8093E8006AE270E0CE0101960E941C
:102F1000681FB5C08091440290914502432F552708
:102F200043305105A9F068F44130510509F40DC151
:102F30004230510509F0FAC084E790E0EAEDF3E091
:102F40004BC04132510529F14232510589F1EEC0A1
:102F5000C901992781309105A1F058F0029709F035
:102F6000E5C0E0E6F4E0E4918E2F90E0E0E6F4E0E6
:102F700030C0ECE9F4E0E4918E2F90E0ECE9F4E06D
:102F800028C0E6E8F4E0E4918E2F90E0E6E8F4E073
:102F900020C08430910508F0C9C0880F991FFC013A
:102FA000ED5BFE4F0190F081E02D89E090E014C0D0
:102FB0008430910508F0BAC0FC01EE0FFF1FE55CFC
:102FC000FE4F0190F081E02DDC01A95CBE4F8C9199
:102FD00090E0009709F4AAC02091E800277F209391
:102FE000E80020914602309147028217930708F4C7
:102FF0009C0140E02115310589F180913E02882332
:1030000009F43DC08530D9F18091E80083FD37C0D7
:103010008091E80082FD2FC08091E80080FFEACF18
:103020004091F3008091F20090E0942B211531053E
:1030300059F08830910540F444914093F100319665
:10304000215031090196F2CF41E0089709F040E0A4
:103050008091E8008E778093E800CCCF4111CDCFEE
:103060000AC080913E02882351F0853041F0809162
:10307000E80083FD04C08091E80082FFF2CF8091D8
:10308000E8008B778093E80051C0803809F04EC08B
:103090008091E800877F8093E80080913F028093D1
:1030A000F1008091E8008E77D2CE81113FC08091EF
:1030B00042029091430299270297C4F58091E8005B
:1030C000877F8093E8001091420210933F020E9494
:1030D000141F111106C08091E30087FD02C081E03A
:1030E00001C084E080933E0242E061EC81E00E94F6
:1030F000331F42E261EC84E00E94331F42E261EC44
:1031000082E00E94331F42E260EC83E00E94331FA2
:1031100042E261EC85E00E94331F80913E028430E0
:1031200011F081E001C082E0809311018091E800FC
:1031300083FF10C08091E800877F8093E800809132
:10314000EB0080628093EB0005C082E190E0EEE44A
:10315000F4E042CFAA96E3E00C94C82C1F920F92A1
:103160000FB60F9211242F933F934F935F936F935A
:103170007F938F939F93AF93BF93CF93DF93EF93FF
:10318000FF93C091E900CF708091EC00D82FD170EF
:1031900080FDD0E81092E9008091F000877F809355
:1031A000F00078940E94D2151092E9008091F0000E
:1031B00088608093F000CD2BCF70C093E900FF9121
:1031C000EF91DF91CF91BF91AF919F918F917F91BF
:1031D0006F915F914F913F912F910F900FBE0F9084
:1031E0001F901895E8EDF0E080818E7F808310922B
:1031F000E2001092DA001092E100A0EEB0E08C91B3
:1032000081608C9380818F77808319BCA7EDB0E0BB
:103210008C918E7F8C9380818F7E8083109233027D
:103220000895A0E0B0E0E7E1F9E10C94A72CC8ED27
:10323000D0E088818F7E8883E7EDF0E08081816037
:10324000808384E082BF81E08093330288818E7F17
:10325000888302EE10E0F80110821092DA0081EE0D
:10326000C82ED12CF601108288818F7788838881BF
:103270008068888388818F7D888319BC10923E0284
:1032800010923F0210923D0210923C0290EEE92E05
:10329000F12CF70180818B7F808388818160888316
:1032A00042E060E080E00E94331FF60180818E7F63
:1032B0008083F80180818160808380818860808341
:1032C000F70180818E7F8083888180618883CDB77C
:1032D000DEB7E8E00C94C32C1F920F920FB60F924A
:1032E00011242F933F934F935F936F937F938F930B
:1032F0009F93AF93BF93EF93FF938091E10082FF81
:1033000049C08091E20082FF45C08091E1008B7F3F
:103310008093E100209132022F5F822F62E30E94AE
:103320003F2C992319F02093320234C010923202BC
:1033300080913102882371F180913E02843041F501
:103340008091E9008F702091EC00922F917020FD08
:1033500090E8892B95E09093E9009091EB0090FF25
:1033600014C09091EE0097FF10C09091E80095FF77
:1033700003C01092F100F9CF9091E80090FF05C0D2
:103380009091E8009E779093E8008F708093E90019
:10339000109231028091DA0080FF2AC08091D8001B
:1033A00080FF26C08091DA008E7F8093DA008091C2
:1033B000D90080FF18C080E189BD82E189BD09B4D0
:1033C00000FEFDCF81E080933E02809133028111A7
:1033D0000FC00E94F2180E9411198091E2008460CF
:1033E0008093E20005C019BC10923E021092330295
:1033F0008091E10080FF1AC08091E20080FF16C03A
:103400008091E2008E7F8093E2008091E2008061F3
:103410008093E2008091D80080628093D80019BC2C
:1034200085E080933E0283E0809311018091E1006A
:1034300084FF37C08091E20084FF33C080E189BD02
:1034400082E189BD09B400FEFDCF8091D8008F7D57
:103450008093D8008091E1008F7E8093E10080917D
:10346000E2008F7E8093E2008091E2008160809391
:10347000E20080913F02882311F084E007C0809130
:10348000E30087FD02C081E001C083E080933E023B
:1034900080913E02843011F081E001C082E080938F
:1034A00011018091E10083FF2CC08091E20083FF35
:1034B00028C08091E100877F8093E10082E08093C3
:1034C0003E0210923F028091E1008E7F8093E100E6
:1034D0008091E2008E7F8093E2008091E200806123
:1034E0008093E20042E060E080E00E94331F809120
:1034F000F00088608093F00081E080931101809358
:103500001001FF91EF91BF91AF919F918F917F91AA
:103510006F915F914F913F912F910F900FBE0F9040
:103520001F9018952091E4003091E50095E64091B8
:10353000EC00842F817040FF23C08091E80080FD63
:103540001DC080913E02882399F0853099F08091CA
:10355000EB0085FD11C04091E4005091E500241777
:10356000350729F3915011F09A01E1CF84E00895D5
:1035700082E0089583E0089581E0089580E0089551
:103580004091E80042FFDDCF0895FC01EE0FFF1FE0
:103590008E0F9F1FFC01E653FD4F61834083228302
:1035A0000895269A0895089585B18F7B95B190640A
:1035B0002FB7F894EAECF2E033E0E231F30789F058
:1035C000319148E095B9000000C037FF85B9330F4D
:1035D000000000C000C000C085B900C04A9591F746
:1035E000EBCF2FBF8FE594E00197F1F700C000000B
:1035F0000895A0E0B0E0EFEFFAE10C94A22CFC01FA
:103600008280748081E08483E0EAF4E09490EFE1CA
:10361000F5E0E4910091C5020695015810E0000F15
:10362000111F012F1127CAE4D2E0C12CD12CAA24EA
:10363000AA94B12CE919EE2EF12C22E0281530F0D5
:103640008091C30288838091C4028983711003C072
:103650001B821A824AC08B818823F9F081508B83A8
:103660002FEF829FC00111246C8170E00E94592CC1
:10367000FB01FF27E056FB4F8491E82FE9192FEF5C
:10368000E29FC0011124B7010E94592C8091C5020C
:10369000689FB00111247A8328C00E94742BB50161
:1036A0000E946D2C8017910704F582E0881588F43C
:1036B0000E94742BB5010E946D2C88830E94742B8C
:1036C0002091C4022695622F70E00E946D2C280F75
:1036D00029831A828091C502843120F0893C18F038
:1036E00088EC01C084E18C838B834A814A3B08F0DB
:1036F00049EB9601698188810E9448282FEFC21A00
:10370000D20A259688E1C816D10409F096CF0E9406
:103710008927CDB7DEB7EDE00C94BE2C0F931F9335
:10372000CF93DF938C01C0E0D0E0F8018481CC30EE
:10373000D1051CF4882351F002C0811107C04091CB
:10374000C5024A3B08F049EB9E0102C09E0140E0E1
:103750006091C4028091C3020E9448282196C8311A
:10376000D10519F70E948927F801848190E001961C
:10377000817099278483DF91CF911F910F910895D4
:10378000A0E0B0E0E6ECFBE10C94A32CEC014C8152
:10379000042F10E09801D8010E94302C9B01AC014D
:1037A0000E94FB2B6B017C01E0E2F0E0E01BF10BDF
:1037B000A5E5B0E09B01AC010E94FB2B4B015C0135
:1037C0009F01DF010E948E2C9B01AC010E94062C00
:1037D0009B01AC012C0D3D1D4E1D5F1DC501B401AB
:1037E0000E940E2C822F022F2A3228F493E0299F68
:1037F000900111240DC025E530E0281B3109C901D5
:10380000880F991F280F391F37FF02C02F5F3F4FC6
:1038100035952795122F1095E12CF12C85E5D82EA2
:10382000D01AE1FC02C08D2D01C0802F412F1A3B20
:1038300008F049EB97016091C4020E9448288FEF7D
:10384000E81AF80A98E1E916F10459F70E94892765
:103850008C81811102C091E003C0803219F49FEF86
:103860009093140190911401890F8C83CDB7DEB72A
:10387000ECE00C94BF2CCF93DF93C0E0D0E020E0CD
:1038800040E060E0CE010E94C51A2196C831D10502
:10389000B1F7C0E0D0E080914902082E000C990BEE
:1038A000C817D907ACF080911301082E000C990BB2
:1038B0008C179D076CF04091C5024A3B08F049EB1C
:1038C0009E016091C4028091C3020E94482806C0F4
:1038D00020E040E060E0CE010E94C51A2196C83188
:1038E000D105C9F60E948927809112019091490261
:1038F000980F9093490220911301280F20931301F0
:10390000121614F497311CF0819580931201DF9107
:10391000CF910895A0E0B0E0E0E9FCE10C94A82C80
:10392000FC01828180FF03C0FF24FA9402C0FF24BF
:10393000F394C0E0D0E098E1D92E20E040E060E0D0
:10394000CE010E94C51A04E010E0E12C80914802EB
:103950008E0D89312CF06D2D0E944B2C892F02C0C9
:1039600087FD885E082E000C990BC817D907A9F4AB
:103970008091C502809FA001819F500D1124559513
:103980004795559547954A3B08F049EB9E01609154
:10399000C4028091C3020E944828EF0C0150110913
:1039A000A9F62196C831D10541F60E948927809158
:1039B0004802F1E0FF1206C0811102C087E107C092
:1039C000815005C090E00196BE010E946D2C80934D
:1039D0004802CDB7DEB7E7E00C94C42CEF92FF921B
:1039E0001F93CF93DF93EC0110E0E12CF12C409179
:1039F000C5024A3B08F049EB8C8197016091C402F3
:103A0000810F0E9448288FEFE81AF80A165F103FCE
:103A100071F70E9489279A818C8190FF02C08F5F85
:103A200001C081508C83DF91CF911F91FF90EF9067
:103A30000895CF93DF93EC014091C5029C8190FFE4
:103A400002C0842F01C080E091FF02C0642F01C03A
:103A500060E092FF40E00E94A1278C8190E00196F7
:103A6000877099278C83DF91CF910895CF93DF934F
:103A7000EC01E2ECF2E0438162818C810E94C0277C
:103A80008C818F5F8C83DF91CF910895CF93DF93EB
:103A9000EC01EC81F0E0E056FB4F4491E2ECF2E007
:103AA000628181810E94C0278C818F5F8C83DF912E
:103AB000CF9108951F93CF93DF93962F8730E8F42B
:103AC0006530D8F44C30C8F4632F122FC42FD0E0E7
:103AD000CC0FDD1F28E1929FC00DD11D112498E766
:103AE000899FC00DD11D1124CE0188960E94A82B5C
:103AF000612FCE0189960E94A82BDF91CF911F9153
:103B000008950F931F93CF93DF93873008F56530A7
:103B1000F8F44C30E8F4C42FD0E0CC0FDD1F28E1DE
:103B2000629FC00DD11D112438E7839FC00DD11DA8
:103B30001124CE0188960E94842B90E0182F002734
:103B4000CE0189960E94842B9801282BC90102C0BE
:103B500080E090E0DF91CF911F910F91089589321D
:103B600089F1F0F4843171F1B0F4873009F077C055
:103B700081E08093160184E1809315018AE08093AF
:103B800018018EE18093170188E080931A0188E282
:103B90008093190164C092EE980F9A30F0F05FC0E4
:103BA000803509F444C028F48F3409F058C08AE005
:103BB0003FC0813529F0823509F051C081E038C01D
:103BC0008FEF36C080911603882379F11092160387
:103BD000109215031092140342C08D518093160366
:103BE000833099F038F4813069F08230D9F485E17E
:103BF00091E00DC0853099F078F0863099F489E134
:103C000091E005C086E191E002C088E191E09093E7
:103C100015038093140323C087E191E0F8CF8AE174
:103C200091E0F5CF109216031AC080E0089586EF58
:103C3000E0911403F0911503309789F02081082E4C
:103C4000000C990B820F911D8F3F910519F014F014
:103C50008FEF04C097FF02C0108201C0808381E013
:103C60000895482F50E0FA013597EF33F10508F039
:103C700073C0ED54FF4F0C94812C0E943A266AC009
:103C800080911303817F8E7F8093130381E0809363
:103C9000120308950E9429142FEF84E39CE0215021
:103CA00080409040E1F700C000000E942D2052C0EB
:103CB00080911303982F9095917090FB80F98093D9
:103CC0001303911147C0897F877F10C08091130330
:103CD00081FB222720F991E0922790FB81F98093C4
:103CE00013039923B9F18091130381608093130327
:103CF00031C08091130382FB222720F991E09227A3
:103D000090FB82F9ECCF8091130383FB222720F9EB
:103D100091E0922790FB83F9E2CF0E9429148091D1
:103D2000550387FB222720F991E0922790FB87F922
:103D3000809355030FC0895301C08D5191E001C09C
:103D4000990F8A95EAF7892F01C081E00E94261415
:103D50000E94291481E0089580E0089580910F0168
:103D600008959FB7F894109231029FBF90913E0240
:103D7000943009F057C09091E9009F703091EC00A9
:103D8000232F217030FD20E8922B25E02093E900BD
:103D90002091EB0020FF43C02091EE0027FF3FC0A1
:103DA00020915C03222321F02091E80025FF37C0F9
:103DB00010925C0326E03091E80035FD15C030918B
:103DC0003E02343061F53091EB0035FD28C02150C2
:103DD00021F481E080935C0322C0EFE9FFE031979A
:103DE000F1F700C00000E7CF8093F1008091E80078
:103DF00085FD0AC08091E80080FFFCCF8091E8003B
:103E00008E778093E80006C08FB7F89421E0209366
:103E100031028FBF9F709093E90080E008959F70FA
:103E20009093E9008FEF08958091400287FF11C0C1
:103E30008091E80082FD05C080913E028111F8CF9B
:103E400011C08091E8008B770BC080913E028823DF
:103E500049F08091E80080FFF8CF8091E8008E77EC
:103E60008093E8000895982F973068F59093E900C3
:103E7000981739F07091EC002091ED005091F0000E
